:10000000122AFF3FFF3FFF3F3E30031383129C0045
:100010006123400897009601170816020318AC28C0
:100020000B108B158B13630016089C00612340088E
:100030009800F0300605C2004208F03A0319A128E2
:10004000F0300605C200420899004208703A031DCC
:100050002B28990184281908B03A031D3228013051
:10006000990084281908D03A031D392802309900D4
:1000700084281908E03A031D402803309900842899
:100080001908C03A031D79289722990104301902F2
:100090000318782803301905C0004008C200013059
:1000A000C000420803195828C00D4010FF3F5228D5
:1000B000400885009701C830170203187628F030F1
:1000C0000605C2004208F03A031973288501190A8F
:1000D000C000400894003F309A0040089B00F42282
:1000E0009722C00108003223970A5B28990A462804
:1000F00045281908303A031D84280F3085009722BF
:1001000085010230C000080019089C001908063C4F
:10011000C000C101031CC1036C30C00703300318C9
:10012000013FC10740088E0041088D000A088C007D
:1001300074239D000C088A0001309E009F01092154
:10014000192832235921190818060319AA281F2330
:10015000C0010800960A0C280130C00008000313F3
:100160008312CD01C901C8014108400403190034BC
:1001700041084506CA00CA1BCD09CB01C51FC528C9
:10018000C409C509C40A0319C50AC11FCC28C0097E
:10019000C109C00A0319C10A41084504CA00CA1BA3
:1001A000E12846224B18F428CD1F0034C009C109AC
:1001B000C00A0319C10AC809C909C80A0319C90A2A
:1001C0000034C51FF028C11BEC284108C9004008B5
:1001D000C800C101C001D428C101C001C00A003457
:1001E000C109C009CB0AD128C80A0319C90A4408A1
:1001F0004802031DD42845084902031DD428C9011B
:10020000C801C00A0319C10AC11FD4280000FF3465
:100210000800031383121C086C3FC000033003184E
:10022000013FC10040088E0041088D000A088C0083
:100230007423A1000C088A0003301C05C00040088C
:10024000C2000130C000420803192A29C00D401025
:10025000FF3F2429400885001E08C0009E03400877
:1002600003194E291D08C0009D03400803194D299C
:1002700001300605C0000130C006003040180130D2
:10028000060601398606A0012108200203184C2920
:1002900000000000A00A442932292C2985010610FB
:1002A0001F08C0009F034008031958293223502912
:1002B0000800031383121308031D632901309C00F7
:1002C00000309D0056230F08C0001008C10011081F
:1002D000C2001208C3006D30C4004E30C500C630E5
:1002E000C6004130C700A0213930C5003030C600FB
:1002F000C701C8014008C50741080318410FC607D8
:1003000042080318420FC70743080318430FC807E2
:100310004708C0004808C1000030C81BFF30C300B8
:10032000FF30C0057F30C1050030C205C30540085D
:100330008F00410890004208910043089200080095
:1003400003138312CD01C31FB229C009C109C20919
:10035000C309C00A0319C10A0319C20A0319C30A4F
:100360008130CD07C71FC029C409C509C609C709FF
:10037000C40A0319C50A0319C60A0319C70ACD0A14
:10038000DB214D1CDA29C009C109C209C309C8090A
:10039000C909CA09CB09C00A0319C10A0319C20A4B
:1003A0000319C30A0319C80A0319C90A0319CA0A97
:1003B0000319CB0A0800031383122230CC00C801B2
:1003C000C901CA01CB01CC030319112A0310CB0CBC
:1003D000CA0CC90CC80CC30CC20CC10CC00C031C49
:1003E000E329CC030319032A4408C8074508031866
:1003F000450FC90746080318460FCA0747080318E0
:10040000470FCB07E7294408C80745080318450FDD
:10041000C90746080318460FCA0747080318470FBD
:10042000CB07080003138316850183128501F03082
:1004300083168600831286017F30831681053F3044
:100440009C006123400894000C239722B8220313D8
:100450008316D922400803193B2A4423042040086C
:1004600095004008003A03192D2A1508023A03198D
:100470003B2A9722272A1508013A031D442A0C23F8
:100480000C230C230C239722262A452A03138312BC
:10049000410DC80DC90D4408C8024508031C450F8D
:1004A000C902C00DC10D0F30CC00410DC80DC90DE2
:1004B0004408401C612AC8024508031C450FC902B4
:1004C000662AC80745080318450FC907C00DC10DA6
:1004D000CC0B552A4018722A4408C807450803184F
:1004E000450FC90700000800031383121A089C0077
:1004F000612340089C004008063CC000C101031C69
:10050000C1036C30C00703300318013FC107400826
:100510008E0041088D000A088C0074239D000C0891
:100520008A0014089E000A309F00092108000B3041
:1005300003138312CC00FF30CB00FF30CA00CC0B7A
:10054000A22AA92ACB0BA52AA82ACA0BA52AA22A25
:100550009F2A3330CB00FF30CA00CB0BB02AB32A1E
:10056000CA0BB02AAD2A8830CA00CA0BB52A0800C7
:10057000031383129601031383123E3016020318ED
:10058000D22A59210430C4000030C500AF204808E9
:10059000C0004908C10040089B0016089A00F422D8
:1005A000960ABB2A031383163E309A009B01F4225D
:1005B00008003E30031383129C006123400896001C
:1005C000400A960016083E3A031DE82AC0010800BA
:1005D00032238B110B103E309A0016089B00F42238
:1005E00032230130C0000800000003138316881C6A
:1005F000FB2A0000F52A1A08831289001B088800CC
:100600008316881308158B1355308900AA3089008A
:1006100088148B1708110800073003138312960003
:100620001608003C03181E2B16039C0032309D0058
:1006300001309E009F0109219603102B080003132F
:1006400083129A0107301A020318302B1A089C00F3
:1006500032309D0001309E009F0109219A0A222B11
:10066000972208001A3003138312CB00FF30CA0010
:10067000CB0B3B2B3E2BCA0B3B2B382BE730CA0056
:10068000CA0B402B000008003E30031383129C006D
:100690006123400897009601170816020318552B8E
:1006A00016089A007422960A4C2B08000313831232
:1006B0001C088F001D0890009101920101309300E9
:1006C0000800031383121C0889008316881308147A
:1006D00083120808C000080084349434A534B03470
:1006E000C634DC34F7340800031383120D088A0083
:1006F0000E0882000800FF3FFF3FFF3FFF3FFF3F24
:10420000FF00FF00FF00FF00FF00FF00FF00FF00B6
:10421000FF00FF00FF00FF00FF00FF00FF00FF00A6
:10422000FF00FF00FF00FF00FF00FF00FF00FF0096
:10423000FF00FF00FF00FF00FF00FF00FF00FF0086
:10424000FF00FF00FF00FF00FF00FF00FF00FF0076
:10425000FF00FF00FF00FF00FF00FF00FF00FF0066
:10426000FF00FF00FF00FF00FF00FF00FF00FF0056
:10427000FF00FF00FF00FF00FF00FF00FF00040041
:10428000FF00FF00FF00FF00FF00FF00FF00FF0036
:10429000FF00FF00FF00FF00FF00FF00FF00FF0026
:1042A000FF00FF00FF00FF00FF00FF00FF00FF0016
:1042B000FF00FF00FF00FF00FF00FF00FF00FF0006
:1042C000FF00FF00FF00FF00FF00FF00FF00FF00F6
:1042D000FF00FF00FF00FF00FF00FF00FF00FF00E6
:1042E000FF00FF00FF00FF00FF00FF00FF00FF00D6
:1042F000FF00FF00FF00FF00FF00FF00FF00FF00C6
:10430000FF00FF00FF00FF00FF00FF00FF00FF00B5
:10431000FF00FF00FF00FF00FF00FF00FF00FF00A5
:10432000FF00FF00FF00FF00FF00FF00FF00FF0095
:10433000FF00FF00FF00FF00FF00FF00FF00FF0085
:10434000FF00FF00FF00FF00FF00FF00FF00FF0075
:10435000FF00FF00FF00FF00FF00FF00FF00FF0065
:10436000FF00FF00FF00FF00FF00FF00FF00FF0055
:10437000FF00FF00FF00FF00FF00FF00FF00FF0045
:10438000FF00FF00FF00FF00FF00FF00FF00FF0035
:10439000FF00FF00FF00FF00FF00FF00FF00FF0025
:1043A000FF00FF00FF00FF00FF00FF00FF00FF0015
:1043B000FF00FF00FF00FF00FF00FF00FF00FF0005
:1043C000FF00FF00FF00FF00FF00FF00FF00FF00F5
:1043D000FF00FF00FF00FF00FF00FF00FF00FF00E5
:1043E000FF00FF00FF00FF00FF00FF00FF00FF00D5
:1043F000FF00FF00FF00FF00FF00FF00FF00FF00C5
:02400E00FA3F77
:00000001FF
